:100000000C94BE020C94F6020C94F6020C94F602C8
:100010000C94F6020C94F6020C94F6020C94F60280
:100020000C94F6020C94F6020C947F280C9451293F
:100030000C945E230C94F6020C94F6020C94F602D7
:100040000C94F6020C945D1E0C94F6020C94F602CD
:100050000C94811E0C94E6230C94F6020C94F60288
:100060000C94F6020C94F6020C94F6020C94F60230
:100070000C94F6020C94F6020C94F6020C94F60220
:100080000C94F6020C94F6020C94F6020C94F60210
:100090000C94F6020C94F6020C94F6020C94F60200
:1000A0000C94F6020C94F6020C94F602C605C605F2
:1000B000F205F2055A0678069007900783061C079A
:1000C0002D072D07BE29E529DD2AE529DD2A312A5C
:1000D000542ADD2AAB2ABA2A165C1E001F00200013
:1000E00021002200230024002500260027002D00E7
:1000F0002E002A002A002B0014001A000800150008
:1001000017001C0018000C00120013002F00300014
:1001100031004600015104001600070009000A00E2
:100120000B000D000E000F0033003400280000000B
:100130004C00E10035001D001B0006001900050001
:1001400011001000360037003800E50052004B0067
:100150000000E000E300E2002C4100002C00000061
:10016000E6000151E400500051004F004E00350000
:100170003A003B003C003D003E003F004000410093
:1001800042004300440045004C004C00390001008F
:100190005200010001000100010001000100005CAB
:1001A0004600470048000100C35C010050005100B8
:1001B0004F00010001000100010001000100CB5CC3
:1001C000CA5C49000000C45CE1000100AC00AE0064
:1001D000AB000100010001000100A800AA00A90075
:1001E0000100C65C4A000000E000E300E2000100FC
:1001F000000001000000010001000100C95CC75CB3
:10020000C85C4D0000047F3F1F64321464321478D0
:100210003C1E1E140A052223252628292A2C2D2FB0
:100220003032333536383A3B3D3E4042434547490C
:100230004A4C4E5051535557595A5C5E6062646641
:1002400068696B6D6F71737577797B7D7F8183854D
:1002500087898A8C8E90929496989A9C9E9FA1A34F
:10026000A5A7A8AAACAEAFB1B3B4B6B8B9BBBCBE73
:10027000BFC1C2C3C5C6C7C9CACBCCCDCED0D1D2EF
:10028000D2D3D4D5D6D7D7D8D9D9DADADBDBDBDCF1
:10029000DCDCDCDCDDDDDDDDDCDCDCDCDCDBDBDB9D
:1002A000DADAD9D9D8D7D7D6D5D4D3D2D2D1D0CEFD
:1002B000CDCCCBCAC9C7C6C5C3C2C1BFBEBCBBB902
:1002C000B8B6B4B3B1AFAEACAAA8A7A5A3A19F9E80
:1002D0009C9A98969492908E8C8A89878583817F48
:1002E0007D7B79777573716F6D6B69686664626029
:1002F0005E5C5A5957555351504E4C4A49474543F5
:1003000042403E3D3B3A3836353332302F2D2C2A91
:10031000292826252322FFAA7F554000010101013B
:1003200001010101010202020202020202020303B0
:100330000303030303030404040404040405050580
:100340000505060606060607070707070808080842
:10035000090909090A0A0A0B0B0B0C0C0C0D0D0DEF
:100360000E0E0E0F0F0F1010111111121213131485
:1003700014151516161717181819191A1A1B1B1CFD
:100380001D1D1E1E1F202021222223242425262657
:10039000272829292A2B2C2D2D2E2F30313232338C
:1003A0003435363738393A3B3C3D3E3F4041424395
:1003B0004445464748494A4C4D4E4F505153545579
:1003C0005658595A5B5D5E5F616264656668696B29
:1003D0006C6D6F7072737577787A7B7D7E808283A7
:1003E0008587888A8C8E8F91939596989A9C9EA0EB
:1003F000A2A3A5A7A9ABADAFB1B3B5B7BABCBEC0F8
:10040000C2C4C6C9CBCDCFD1D4D6D8DBDDDFE2E4C0
:10041000E7E9EBEEF0F3F5F8FAFDFF0A03430041DC
:10042000003600360000000C0342006100720072CA
:1004300000790000000403090409023B00020100E6
:10044000A0FA0904000001030101000921110100C3
:100450000122400007058103080001090401000191
:100460000300000009211101000122B600070582E6
:1004700003200001120100020000000857546060D0
:1004800001000102000105010902A1018502090123
:10049000A100050919012908150025019508750114
:1004A00081020501093009311581257F9502750802
:1004B000810609381581257F950175088106050C8F
:1004C0000A38021581257F950175088106C0C0058F
:1004D000010980A101850319012AB700150126B77A
:1004E00000950175108100C0050C0901A10185046A
:1004F00019012AA002150126A0029501751081009C
:10050000C005010906A1018506050719E029E715BF
:100510000025019508750181020507190029EF15CD
:1005200000250195F075018102050819012905953D
:100530000575019102950175039101C00501090638
:10054000A101050719E029E71500250195087501A6
:1005500081029501750881010507190029FF150021
:1005600026FF0095067508810005081901290595E3
:100570000575019102950175039101C011241FBEFB
:10058000CFEFDAE0DEBFCDBF04B603FE18C0809126
:10059000210390912203A0912303B091240387307B
:1005A000904BA740B04B59F41092210310922203B4
:1005B0001092230310922403E0E0F8E3099511E080
:1005C000A0E0B1E0E0E4F8E502C005900D92A83C9F
:1005D000B107D9F723E0A8ECB1E001C01D92A13228
:1005E000B207E1F70E94A2130C941E2C0C94000099
:1005F00081E0089581E008950C94FA0208950C9426
:10060000FE021F93CF93DF9300D000D01F92CDB78F
:10061000DEB749835A836B833091CB0189819A81FC
:10062000311114C0662359F0222349F00E94CD09EC
:10063000182F682F89819A810E94760903C00E9431
:10064000A109182F69817A81812F04C00E94CD09E8
:1006500069817A810F900F900F900F900F90DF912A
:10066000CF911F910C940D11FC01262F40815181D7
:100670006281738184810C94010381E00895CF939A
:10068000DF93EC0160E00E943403BE01DF91CF9163
:100690000C94FF020C9453120C944F1208950E9474
:1006A00020080E944E032FEF84E39CE021508040FD
:1006B0009040E1F700C000000C940C240F931F93AE
:1006C000CF93DF938C0161E00E943403EC01B80109
:1006D0000E94FC02882309F44BC0B801CE010E949D
:1006E000261E882309F444C0B801CE010E94A92126
:1006F0008823F1F1B801CE010E94BD1F8823C1F10A
:10070000B801CE010E940521882391F1B801CE01E4
:100710000E946A1C882361F1F8018281882309F113
:10072000CB358DE5D807C1F050F4C115FCE5DF07E6
:1007300081F0CF3DDC45A9F40E94040F19C0CC35EF
:10074000EDE5DE0761F0CD35DD4559F40E94470E39
:1007500008C00E944F030CC00E94500E02C00E94AD
:10076000530EC801DF91CF911F910F910C94F802A5
:1007700080E0DF91CF911F910F9108950E94402357
:1007800080E00E94B61E0C94E9030E944A1D0E945C
:10079000EC030C94462308950C94CB0381E0089558
:1007A000CF93C82F0E94CE03882329F0C1FF02C037
:1007B000599A01C05998CF910895519A599808951E
:1007C000CF93C82F0E94CC038C2F0E94D003CF91CF
:1007D000089580E00C94E0030E9405220C94E0034D
:1007E0000E9405229091CA01891721F08093CA01C5
:1007F0000C94E0030895CF93DF93CDB7DEB72B972A
:100800000FB6F894DEBF0FBECDBF4F835887698700
:100810007A878B8761110E94930D9E012F5F3F4F56
:1008200086E0F90111928A95E9F785E0FE01379695
:10083000D90101900D928A95E1F789819A814C81C5
:100840005D81452B31F09F3F31F491E08F3F19F4EA
:1008500003C091E001C090E090FF09C049815A8136
:100860006B817C818D819E810E94B40C05C0C90181
:100870000E943D038111F2CF2B960FB6F894DEBF94
:100880000FBECDBFDF91CF910895FC018081918192
:100890000E940F0A0895CF93882309F4A4C0C82F9B
:1008A0008238C1F40E94052281FD9DC069E38091D8
:1008B0000201909103010E94FB220E94B50D2FEFCF
:1008C00081EE94E0215080409040E1F700C00000AC
:1008D00069E319C0833801F50E94052280FD83C0B9
:1008E00063E580910201909103010E94FB220E9426
:1008F000B50D2FEF81EE94E0215080409040E1F75C
:1009000000C0000063E580910201909103010E9404
:100910000623CF910C94B50D8438C1F40E940522B2
:1009200082FD61C067E480910201909103010E9401
:10093000FB220E94B50D2FEF81EE94E02150804004
:100940009040E1F700C0000067E4DDCF8CEF8C0F32
:10095000813AD0F46C2F80910201909103010E94A2
:100960007B22882349F06C2F809102019091030132
:100970000E9406230E94B50D6C2F80910201909178
:1009800003010E94FB22C5CF80E28C0F883048F41F
:10099000C77081E001C0880FCA95EAF70E94760D02
:1009A000B8CFEBE5EC0FE33040F4F0E0E65AFE4F51
:1009B000808190E0CF910C943922E8E5EC0FE7318B
:1009C00050F4F0E0EE0FFF1FE45DFE4F8081918157
:1009D000CF910C944F22CD3E30F08C2F0E942714E3
:1009E000CF910C94F914CF910895882309F464C031
:1009F000823879F40E94052281FF5EC069E380910C
:100A00000201909103010E94FB220E94B50D69E34F
:100A100010C08338B1F40E94052280FF4DC063E509
:100A200080910201909103010E94FB220E94B50D6A
:100A300063E580910201909103010E9406230C94CA
:100A4000B50D843879F40E94052282FF35C067E431
:100A500080910201909103010E94FB220E94B50D3A
:100A600067E4E7CF9CEF980F913A10F4682FE1CF3D
:100A700090E2980F983050F4877091E001C0990F80
:100A80008A95EAF7892F0E947C0DD9CF9BE5980FB4
:100A9000933020F480E090E00C94392298E5980F90
:100AA000973120F480E090E00C944F228D3E20F0AE
:100AB0000E9482140C94F91408951F93CF93DF932E
:100AC000182FEB010E944B04209741F08FE99FE023
:100AD0000197F1F700C000002197F6CF812FDF9139
:100AE000CF911F910C94F504893319F060E070E008
:100AF00002C060E570E00C945D05882321F00E943F
:100B0000760D0C94B50D0895882321F00E947C0D7C
:100B10000C94B50D0895CF92DF92EF92FF920F9350
:100B20001F93CF93DF937C01D62FC72FFC01128137
:100B3000058102950F700E946C0D8823B9F0112376
:100B4000A9F08C2F807F803421F080E28D0F8830D7
:100B500068F08091E30282FD09C082E00E94150ED8
:100B60000E946C0D91E0D82ED92601C0D12CCC2E3C
:100B7000C2948FE0C8228C2D90E08C30910508F053
:100B8000CFC1FC01EA5AFF4F0C94792B8C2F807F48
:100B9000CF70882311F0C295C07F112399F0CC2328
:100BA00009F4AAC180E28D0F883010F0D11104C081
:100BB0008C2F0E94760D03C08C2F0E94860D0E9400
:100BC000B50D9AC18D2F0E94F504CC2309F4A8C15C
:100BD00080E28D0F883038F1DD2329F18C2F0E94BF
:100BE0008C0D24C08C2F807FCF70803211F0C29585
:100BF000C07FDD2319F0D130A1F13DC08091E30227
:100C000082FF17C0112349F0CC2329F08C2F0E94BA
:100C1000760D0E94B50D80E070C180E00E94F50461
:100C2000CC2309F47DC18C2F0E947C0D0E94B50D50
:100C300077C1112371F0002341F0013031F40E949B
:100C4000960D8C2B0E949E0D6BC10E94960D8C2BD5
:100C50001DC0002319F0013009F462C10E94AB0DE0
:100C600025C0112321F0063008F05AC10EC005300E
:100C700008F056C11BC0112361F0002331F0F701C9
:100C8000858180FF39C18F7085838C2F0E947D05FF
:100C900047C1002359F0D93309F03FC1FFEF07EEF8
:100CA00013E0F15000401040E1F735C18C2F0E9455
:100CB000840536C18C2F86958695837019F0813016
:100CC00061F02EC1112321F08D2F9C2F937002C053
:100CD00080E090E00E9439222BC1112321F08D2F5A
:100CE0009C2F937002C080E090E00E944F2220C1B0
:100CF0008D2F112319F00E94271402C00E94821424
:100D00000E94F91415C18C2F837009F047C011118E
:100D10000BC12D2F229526952770220F220F6D2FA4
:100D20006F70862F90E0A0E0B0E0022E04C0880F24
:100D3000991FAA1FBB1F0A94D2F7D4FF10C04FE01F
:100D400050E060E070E004C0440F551F661F771F3D
:100D50002A95D2F7409550956095709503C040E074
:100D600050E0BA01C695C695C3708A019B01082B55
:100D7000192B2A2B3B2BC901B801C23049F058F47A
:100D8000C13019F00E948C08CFC00E947A08CCC0F4
:100D90000E949E08C9C00E947808C6C0112319F09D
:100DA0008C2F817001C08695882309F4BDC02D2F3A
:100DB000229526952770220F220F6D2F6F70862F98
:100DC00090E0A0E0B0E0022E04C0880F991FAA1F97
:100DD000BB1F0A94D2F7D4FF10C04FE050E060E090
:100DE00070E004C0440F551F661F771F2A95D2F785
:100DF000409550956095709503C040E050E0BA0171
:100E0000C695C695C3708A019B01082B192B2A2B06
:100E10003B2BC901B801C23049F058F4C13019F078
:100E20000E94510981C00E943F097EC00E9463094F
:100E30007BC00E94B20878C0CF70112339F08C2F8C
:100E40000E94D8088D2F0E947D056EC08D2F0E94B4
:100E500084058C2F0E94F90867C0D23F21F128F445
:100E6000D03F41F0D13FC1F043C0D33F19F1D43F4F
:100E700079F03EC0112341F0053008F051C08C2FAD
:100E80008F710E941E094CC0063008F049C0F7CF90
:100E90008091E30282FF18C0112339F08C2F8F71EB
:100EA0000E94D8083DC01123C9F38C2F8F710E9476
:100EB000F90836C0112329F08C2F8F710E94C308C6
:100EC0002FC00E94BE082CC0112349F0CF718C2F77
:100ED0000E94D80863E08C2F0E94FA0D21C081E0A7
:100EE0000E94150E0230E0F082E00E94150E18C03C
:100EF000112331F0002391F28D2F0E944B0410C07A
:100F0000002399F2D93349F41FEF27EE33E0115053
:100F100020403040E1F700C000008D2F0E94F50412
:100F200088EF8C0D843020F40E9405220E94E0039B
:100F3000DD20C9F00E94680D80FD15C0F701128206
:100F40000E94620D0E94D808C7010E94D4070E9427
:100F5000620DDF91CF911F910F91FF90EF90DF9085
:100F6000CF900C94F908DF91CF911F910F91FF90D2
:100F7000EF90DF90CF9008950F931F93CF93DF935F
:100F8000EC01688179818A810E941A0A8C010E9491
:100F900075090E946608B801CE010E948B05DF9199
:100FA000CF911F910F910895CF93DF93EC0198811A
:100FB00089812B813C81232B31F08F3F31F481E0FB
:100FC0009F3F19F403C081E001C080E080FD1DC097
:100FD000CE010E945E03811110C00E946C0D882317
:100FE000A1F08A81882389F08091E30282FD0DC0FF
:100FF00082E0DF91CF910C94150ECE010E94BC07C8
:10100000CE01DF91CF910C943F03DF91CF910895F2
:1010100080E090E00E94392280E090E00E944F2220
:101020000E94930D0E94B50D0E942A160C94F9148B
:1010300080910201909103010E9411230C940808F1
:101040000E94830D0C94180892959F70963079F049
:1010500010F4925001C09A50923068F4803F69F0C9
:1010600018F4883E40F409C0843F29F406C0883E45
:1010700020F0813F11F080E0089581E00895FC01A7
:10108000808191810E940F0A0E9424080895CF93C5
:10109000DF9300D000D01F92CDB7DEB70F900F9036
:1010A0000F900F900F90DF91CF910895CF93DF9322
:1010B00000D000D000D0CDB7DEB726960FB6F8949A
:1010C000DEBF0FBECDBFDF91CF9108950895089583
:1010D0000C9467080C9468080E946A0860930202E6
:1010E0007093030280930402909305020C94080805
:1010F0000C946C080F931F9300910202109103024D
:101100002091040230910502602B712B822B932BCE
:101110001F910F910C946C080F931F930091020282
:101120001091030220910402309105026023712383
:10113000822393231F910F910C946C080F931F939C
:1011400000910202109103022091040230910502E5
:1011500060277127822793271F910F910C946C08A9
:101160000C9467080E94B0086093FE017093FF0121
:1011700080930002909301020C94080860E070E0F4
:10118000CB010C94B2080F931F9341E050E060E054
:1011900070E08A019B0104C0000F111F221F331F42
:1011A0008A95D2F7C901B8011F910F910C94B2082A
:1011B0000F931F9341E050E060E070E004C0440FE3
:1011C000551F661F771F8A95D2F78091FE01909177
:1011D000FF01A0910002B09101028A019B01082B3E
:1011E000192B2A2B3B2BC901B8011F910F910C948D
:1011F000B2080F931F9341E050E060E070E004C03C
:10120000440F551F661F771F8A95D2F7409550955A
:10121000609570958091FE019091FF01A091000270
:10122000B09101028A019B01082319232A233B2341
:10123000C901B8011F910F910C94B2080F931F932D
:1012400041E050E060E070E004C0440F551F661FAD
:10125000771F8A95D2F78091FE019091FF01A091AE
:101260000002B09101028A019B01082719272A2751
:101270003B27C901B8011F910F910C94B2080F933D
:101280001F930091FE011091FF0120910002309107
:101290000102602B712B822B932B1F910F910C94C9
:1012A000B2080F931F930091FE011091FF0120914E
:1012B00000023091010260237123822393231F9146
:1012C0000F910C94B2080F931F930091FE0110919F
:1012D000FF012091000230910102602771278227CF
:1012E00093271F910F910C94B20808952FE0929FBD
:1012F000800D1124E82FE695E695E695877051E07C
:1013000001C0550F8A95EAF785E0E89FF0011124A6
:10131000E453FE4F20E030E070E04081CB01022E2C
:1013200002C0969587950A94E2F78170819584278B
:101330008523842781932F5F3F4F2530310569F73F
:1013400008952FE0929F800D1124682F6695669571
:101350006695982F977085E0689FB001112440E052
:1013600050E080E0FB01E40FF51FE453FE4F2081C5
:1013700030E0092E02C0369527950A94E2F72170D5
:101380003327042E01C0220F0A94EAF7822B4F5F05
:101390005F4F4530510531F70895BF92CF92DF92EC
:1013A000EF92FF920F931F93CF93DF938C01C09026
:1013B000FE01D090FF01E0900002F09001028091C8
:1013C000020290910302A0910402B0910502C82A82
:1013D000D92AEA2AFB2ACFE1D0E0D701C6010C2E98
:1013E00004C0B695A795979587950A94D2F780FD86
:1013F00004C0219790F7B12C07C0BC2EB8018C2FE8
:101400000E9420110197A9F38B2DDF91CF911F919D
:101410000F91FF90EF90DF90CF90BF900895CF9302
:10142000DF93EC010E94CD09BE010E942011DF91E3
:10143000CF9108951F93CF93DF93EB019091CB0150
:10144000992321F0CB010E940F0A13C0882349F091
:10145000CB010E94CD09182F682FCE010E9476097A
:1014600004C0CB010E94A109182FBE01812F0E9448
:101470002011DF91CF911F9108951F93CF93DF9398
:10148000C091060216E080910702C81799F0D0E0DB
:101490001C9FF0011D9FF00D1124E85FFD4F40815E
:1014A000518162817381848195810E9456082196C1
:1014B000C770E9CFDF91CF911F9108954091380215
:1014C0005091390260913A0270913B0280913C0246
:1014D00090913D020C945608EF92FF920F931F9348
:1014E000CF93DF9380913D0282958F7009F065C0A4
:1014F00080913A02882309F460C080910602F0903E
:101500000702109138020091390260913B027091FC
:101510003C0291E01F3F09F090E0C0910001D091A2
:101520000101292F96E0E92E8F1509F446C06115B7
:10153000710521F00F3F21F030E003C031E001C020
:10154000322F90E030FD36C0E89EF001E99EF00DAC
:101550001124DF01A85FBD4F11963C911197301304
:1015600029C03C91311326C012963C91129731113B
:1015700021C013964D915C911497461B570B4C1745
:101580005D07C0F480913D028F70806180933D02C1
:10159000E35FFD4F80818F708061808388E392E0FC
:1015A0000E94D407DF91CF911F910F91FF90EF9090
:1015B0000C943D0A01968770B7CFDF91CF911F91B0
:1015C0000F91FF90EF9008959F92AF92BF92CF92AC
:1015D000DF92EF92FF920F931F93CF93DF93CDB7DC
:1015E000DEB761970FB6F894DEBF0FBECDBF8C019A
:1015F00085E0F801DE011D9601900D928A95E1F7D4
:10160000D8011296EC9090913802E0913902209125
:101610003B0230913C022115310531F0EF3F31F4AE
:1016200081E09F3F19F403C081E001C080E0B82F42
:10163000B1709B2E80FD47C1D8014C9111965C91F1
:1016400011971396AD90BC90149788E3C82E82E052
:10165000D82EF0903A02B501621B730B2091000165
:1016600030910101FF2009F4D9C080913D02621739
:10167000730708F095C0282F207F09F052C05E1331
:1016800013C0491311C0FE2CE1100EC08F70806191
:1016900080933D020E945E0AC6010E94D407809199
:1016A0003D02F80185834DC1AB2831F05F3F31F435
:1016B00081E04F3F19F403C081E001C080E080FD6C
:1016C00003C081E08E2502C080E090E0F82FF17029
:1016D000FF2E80FF1CC0809106022091070236E099
:1016E000821709F40BC190E0389FF001399FF00D8B
:1016F0001124E85FFD4F6181561306C060814613D7
:1017000003C06281E61203C001968770E9CFFE2C08
:10171000EE2009F416C180913D02816080933D0264
:1017200054C05E1306C0491304C0E11002C0F801A2
:1017300099C0C8010E943F08882361F1EE2051F151
:1017400020913D02822F82958F7090E0029774F075
:10175000809138029091390298878F831986BB86D1
:10176000AA862C87CE0107960E94D40786E0F8014E
:10177000A8E3B2E001900D928A95E1F70E946C0A0D
:101780000E945E0A0AC05E1711F1C8010E943F085C
:1017900081112CC0C8010E94D407FF24F394D1C04A
:1017A000282F207F81F77A2DB98AA88A6E2D898902
:1017B0000E94470888E392E00E94D40786E0D601A1
:1017C0001D928A95E9F70E945E0AF12CBAC049136E
:1017D000DCCFE110DACFF8018583C8010E94D4077D
:1017E00086E0D6011D928A95E9F7ABC0EE2091F212
:1017F00020913D02822F82958F7090E002970CF429
:10180000B5CF80913802909139029A8389831B82E7
:10181000BD82AC822E83CE010196A6CF62177307DC
:1018200008F044C0FE2CEE2009F4B4CF5E1330C0A3
:1018300049132EC020913D0220FD21C0822F8295A8
:101840008F70482F50E041155105C9F0F8012583EC
:101850004F30510541F08F5F982F9295907F822FE6
:101860008F70892B8583C8010E94D40786E0F80118
:10187000A8E3B2E001900D928A95E1F73CC086E0C2
:10188000F801A8E3B2E001900D928A95E1F759C002
:10189000C8010E943F08811169CF80913D0281609B
:1018A00080933D02C8010E94D4074BC07A2DB98AAB
:1018B000A88A6E2D89890E94470886E0D6011D926C
:1018C0008A95E9F718C0EE2009F464CFC8010E9498
:1018D0003F08F82E882309F45DCF86E0F801A8E3DD
:1018E000B2E001900D928A95E1F788E392E00E94C0
:1018F00045040E946C0A0E945E0A23C04D875E87E1
:101900008D859E850E940F0A292F22952F702230E7
:1019100028F49F7039F0811105C00BC0243028F4E1
:101920009F7049F4805E883020F0C8010E94D4077F
:101930009F2CF92C06C0D80115969C91907F91F7A9
:10194000F8CF8F2D61960FB6F894DEBF0FBECDBFD6
:10195000DF91CF911F910F91FF90EF90DF90CF908B
:10196000BF90AF909F9008951F93CF93DF93CDB713
:10197000DEB72C970FB6F894DEBF0FBECDBF4F83F6
:10198000588769877A878B879C87CE0107960E9444
:10199000E40A8823D1F09F8188852A853B85232B03
:1019A00031F08F3F31F481E09F3F19F403C081E0B3
:1019B00001C080E080FD47C04F81588569857A85E8
:1019C0008B859C850E9456083EC086E0FE013796B6
:1019D000DE01119601900D928A95E1F7FF81E8856D
:1019E0006A857B856115710531F0EF3F31F481E047
:1019F000FF3F19F403C081E001C080E080FD23C0F7
:101A00002091070230E0C901019687709927409123
:101A1000060250E084179507F1F1F983EA837D838C
:101A20006C8396E0929FD001939FB00D1124A85F24
:101A3000BD4FFE01319601900D929A95E1F780938A
:101A400007020E943D0A16E080910602909107026B
:101A5000891771F1189FC0011124885F9D4F0E9462
:101A6000E40A882329F1E09106021E9FF001112467
:101A7000E85FFD4F4081518162817381848195814E
:101A80000E9456088091060290E00196877099277F
:101A900080930602D9CF0E9420081092070210926C
:101AA0000602E8E3F2E086E0DF011D928A95E9F79D
:101AB0002C960FB6F894DEBF0FBECDBFDF91CF914D
:101AC0001F91089580915E0285958595859508956D
:101AD00080915E028770089590915E02977081E018
:101AE00009F480E008958091810208959091810227
:101AF000892B80938102089580959091810289239A
:101B0000809381020895109281020895909180023D
:101B1000892B80938002089580959091800289237B
:101B200080938002089510928002089580915F0250
:101B3000089508950C94990D0C949A0D9091E302D8
:101B400092FD08C090915F02981721F080935F0288
:101B50000C949C0D089580915F02882329F01092C7
:101B60005F0280E00C949C0D0895CF93DF93E09189
:101B70000201F0910301809181028083E0910201D2
:101B8000F0910301908180918002892B8083809164
:101B90005F02882381F0E0910201F09103019081BE
:101BA000892B808380910201909103010E9465221C
:101BB00081110E94AB0DC0910201D091030140E25E
:101BC00050E06EE372E0CE010E94C92B892B69F0D0
:101BD00080E2FE01AEE3B2E001900D928A95E1F75A
:101BE000CE01DF91CF910C941122DF91CF91089516
:101BF0000C94990D9091E30292FD10C098E0899F9A
:101C000090011124262B20935E020E94D808809117
:101C10005E028595859585950C94F80D0C94D808F1
:101C200010925E0280E00C94F80D20915E02809587
:101C3000822380935E02982F977099F430E0482FAA
:101C4000082E000C550B2417350759F09091E3022C
:101C500092FD07C08595859585950E94F9080C949D
:101C6000100E08959091E30292FB222720F9281785
:101C700069F080FB92F99093E3028091E2029091E7
:101C8000E3020E94800E82E00C94150E089580916C
:101C9000E30282FB882780F991E089270C94320EB9
:101CA00081E00C94320E80E00C94320E6FEF7FEFE7
:101CB00080E090E00C94082C80E090E00E94E42BFF
:101CC00021E0893E9E4F09F020E0822F089582E0B6
:101CD00090E00C94D62B83E090E00C94D62BCF931D
:101CE00084E090E00E94D62BC82F82E290E00E9410
:101CF000D62B2C2F30E0A901582BCA01CF91089583
:101D0000CF93C92F682F84E090E00E94EA2B6C2FBC
:101D100082E290E0CF910C94EA2BAB01BC018FE002
:101D200090E00C94FC2BAB01BC0183E190E00C949F
:101D3000FC2B60E070E0CB010C94930E60E070E04F
:101D4000CB010E948D0E0C94990E69EE7EEF80E01F
:101D500090E00E94082C60E082E090E00E94EA2B74
:101D600060E083E090E00E94EA2B10920202109261
:101D70000302109204021092050260E084E090E0F9
:101D80000E94EA2B60E082E290E00E94EA2B60E091
:101D900085E090E00E94EA2B60E086E090E00E94FF
:101DA000EA2B6FEF87E090E00E94EA2B40E050E0E2
:101DB000BA0188E090E00E94FC2B60E08DE090E0AA
:101DC0000E94EA2B40E050E0BA0188E190E00E94D6
:101DD000FC2B60E087E190E00E94EA2B40E050E0BD
:101DE000BA018CE190E00E94FC2B60E070E080E2A0
:101DF00090E00E94082C40E050E0BA0188E190E0B9
:101E00000E94FC2B0C949E0E0C94A50E682F8EE065
:101E100090E00C94EA2B0E94CB2360939002709385
:101E20009102809392029093930260938C0270933C
:101E30008D0280938E0290938F02089585B78068FB
:101E400085BF85B7806885BF089581E008950C94AB
:101E5000250F08950C94290F0C94290F0C942C0F26
:101E60000C94290F0C94300F0C94290F0E941E0F14
:101E70008CEF91E10E94FB210E94340F0C94320FF1
:101E80000E942A0F0C94290F0E9416120E94DD0353
:101E90000C94821F0E94B6230E94FB120E94440FE2
:101EA0000E944A1D0E94891B0C942E0F5F926F9214
:101EB0007F928F929F92AF92BF92CF92DF92EF92DA
:101EC000FF920F931F93CF93DF93CDB7DEB72A977F
:101ED0000FB6F894DEBF0FBECDBF0E941013C82E00
:101EE00081110E940B0F32E8832E32E0932E00E026
:101EF00010E0502E802F0E943A125C01F401619094
:101F000071904F016826792661147104B1F40F5F56
:101F10001F4F0530110569F78FEF89838A831B8274
:101F20000E94BF238160782F9D838C8349815A81D1
:101F30006B818D810E94FB033AC08091940281FDE8
:101F40000E944312D12CEE24E394F12CC3018E2184
:101F50009F21892B29F10E94270F8823A9F0DE8277
:101F60005F82AE20BF2081E0AB2809F480E0888743
:101F70000E94BF238160782F9A8789874E815F8175
:101F800068858A850E94FB03000F111FF801EE5738
:101F9000FD4F80819181E826F926F182E08207C019
:101FA000D394EE0CFF1CFFE0DF12D0CFB0CF81E066
:101FB000C11001C080E02A960FB6F894DEBF0FBEB4
:101FC000CDBFDF91CF911F910F91FF90EF90DF90E8
:101FD000CF90BF90AF909F908F907F906F905F90C9
:101FE00008950E94560F0E94BC1B0E94811F0E94F0
:101FF00017150C94F003CF93DF930E942511EC0189
:10200000811521E5920708F045C0811530E5930759
:1020100008F094C0883E910528F5803E910508F0AF
:10202000F8C0883A910570F4853A910508F07CC0B3
:102030008130910509F475C008F4E8C0049708F0F0
:10204000E8C0E4C08F3B910508F0E0C0C85AD0E07A
:10205000CC0FDD1FC35ADE4F0990D881C02DCE01B1
:102060009464D8C0811540E2940758F4811551E07A
:10207000950708F0CEC08D3E910508F4C7C0906565
:10208000C9C0C11580E4D80708F4C0C0DF70CE0114
:10209000906AC0C0811525E59207A8F4811534E542
:1020A000930708F095C0811543E5940708F07BC0BD
:1020B000811552E5950708F061C0D82FCC27CE01D5
:1020C000816F906AA7C0C11589E5D807A0F4C11532
:1020D00028E5D20708F082C0C11536E5D30708F01D
:1020E00095C08C2F0E94B9118F7190E0D82FCC270A
:1020F000CE0190628FC0C1154AE5D40708F474C0C0
:10210000CE0190568115904208F080C08D2F8F71BE
:102110000E94B911DD27D0628F71AE01582BCA0120
:1021200079C081E090E076C0C55AD0E0C557DE4F57
:102130008881C82FD0E0CE0190646CC074E0969581
:1021400087957A95E1F7282F23703C2F337081E033
:1021500090E002C0880F991F3A95E2F79C68AC01A5
:10216000522B9A019C2F9F709695969550E2959FC1
:10217000E0011124C9018C2B9D2B4CC08370992741
:1021800021E030E002C0220F331F8A95E2F79C2F36
:102190009695969580E2989FE0011124C22BD32B4F
:1021A000CE019C6837C08370992721E030E002C0DF
:1021B000220F331F8A95E2F79C2F9695969540E261
:1021C000949FE0011124C22BD32BCE019A6822C028
:1021D000D82FCC27CE01846F906A1CC0DC2FCC276F
:1021E000CE01806F906A16C08C2F8F700E94B9113B
:1021F00094E0D695C7959A95E1F7CF70D0E0DC2FA3
:10220000CC27D0699E01282BC90104C080E090E052
:1022100001C0CE01DF91CF9108952BE4829FC001D0
:102220001124FC012FE0729FE00DF11D1124E60F37
:10223000F11DEE0FFF1FE852FF4F85919491089515
:102240000E940D110E94FB0F08958238910569F1DB
:10225000B0F48133910509F46DC048F489329105D9
:1022600009F463C08A32910509F469C00895853381
:10227000910509F455C089339105B9F00895833E5D
:10228000910569F138F4803E9105B1F0823E9105E7
:1022900009F10895863E9105A9F1873E9105B9F1AE
:1022A000843E910509F064C023C02091E20220FD24
:1022B0004FC021FD4DC008958091E20280FD44C0D1
:1022C0008091E30280FF44C08091E20284FD42C01D
:1022D00083EE4DC08091E20282FF38C0F5CF80913D
:1022E000E20282FD33C08091E30280FD31C0ECCF79
:1022F0008091E30281FF32C08091E20284FD2AC016
:1023000087EE35C08091E20283FF26C0F5CF809131
:10231000E20283FD21C08091E30281FD1FC0ECCF6A
:102320008091E20285FD1CC01DC08091E20285FD06
:1023300019C016C08091E20286FD16C017C08091B8
:10234000E20286FD13C010C089E311C082EE0FC007
:1023500080EE0DC080E00BC086EE09C084EE07C0A1
:1023600089E205C085E303C08AE201C081E390E011
:1023700008959091E20292FF0DC0282F2871283015
:1023800019F4877F846006C0282F2471243011F44B
:102390008B7F886093FF0DC0282F2871283119F496
:1023A000877E846106C0282F2471243111F48B7E2E
:1023B00088612091E30220FF0DC0382F387138303A
:1023C00019F4877F816006C0382F3171313011F4E4
:1023D0008E7F886021FF0DC0282F2871283119F4C5
:1023E000877E816106C0282F2171213111F48E7EF4
:1023F000886194FD877E089580E008950C94560EC0
:102400000E9410138FE39CE90197F1F700C00000D0
:102410000E94101380E00E943A1280FF04C00E94C4
:10242000FE110C940C2408950C9400120E945C0E72
:10243000811102C00E94040F0E94670E80939402D3
:102440000E946F0E9093E3028093E2020E941412A6
:102450000E946B0E682F70E080E090E00E94780888
:102460006091FE017091FF01809100029091010244
:102470000C94B008E82FF0E0EE0FFF1FE251FD4F83
:10248000808191810895089580EA8A95F1F70895F1
:1024900000C008950C94441208950C944C120C94AE
:1024A0004D120C944C120C945112F894E82FE295B2
:1024B000EF70F0E031A1282F2F7081E090E001C093
:1024C000880F2A95EAF7982F9095932391A392A1CC
:1024D000892B82A3789408950F931F93CF93DF9352
:1024E000CDE9D1E089918F3F11F00E94551281E032
:1024F000C23AD807B9F7CEE8D1E00DE911E08991E9
:102500008F3F11F00E9455120C171D07C1F7DF9184
:10251000CF911F910F910895BF92CF92DF92EF92CA
:10252000FF920F931F93CF93DF938C01C62FD0E0C0
:10253000CE0183569E4F6C01FC0190819F3F09F4B0
:1025400050C0B62EF894E92FE295EF70F0E081A12B
:102550009F7021E030E001C0220F9A95EAF7822BAC
:1025600081A382A12095282322A378940E94481257
:10257000EEE8F1E04DE951E021E030E0E12CF12C12
:1025800061916F3F89F0A62FA295AF70B0E0909651
:102590008C9190E06F7002C0959587956A95E2F7EF
:1025A00080FD02C0C90102C080E090E0E82AF92A5B
:1025B000220F331F4E175F0719F7F60180818F3FF7
:1025C00011F00E94551261E0E114F10409F460E099
:1025D0008B2D0E944A12CC0FDD1FC00FD11FF98234
:1025E000E882DF91CF911F910F91FF90EF90DF90E4
:1025F000CF90BF9008950E946C128AE0EEEEF2E058
:10260000DF01982F1D929A95E9F7E4EEF2E0DF01E1
:102610001D928A95E9F785E00E945B130C944A03AA
:10262000FF920F931F93CF93DF93CDB7DEB72A9717
:102630000FB6F894DEBF0FBECDBF8E010F5F1F4FE8
:102640008AE0F80111928A95E9F7F12C6F2DC80103
:102650000E948C12F394F5E0FF12F8CF4AE050E0AC
:10266000B80184EE92E00E94C92BFF24F3940097F6
:1026700009F4F12C892B41F08AE0F801A4EEB2E0D4
:1026800001900D928A95E1F72F2D45E06EEE72E0F4
:1026900084EE92E00E945C130E944C038F2D2A96D8
:1026A0000FB6F894DEBF0FBECDBFDF91CF911F9163
:1026B0000F91FF9008950895FF920F931F93CF936A
:1026C000DF93F82E092F162FD72FC42F222349F07E
:1026D00081E0809397020E94BF239093960280939B
:1026E0009502809197028823D9F08091950290916C
:1026F00096020E94D723059798F0EF2DF02FA12F77
:10270000BD2F80E090E04C2F50E08417950734F403
:10271000219131912D933D930196F7CF109297021D
:10272000DF91CF911F910F91FF9008950E94D725BF
:102730000E944A0F0C94E3250E94E7250E94F10FA6
:102740000C9401260E945D230E94BE250E94360F34
:102750000E9496130E949C130E94400FFBCF809111
:102760009E0280FF06C06091090170E0660F771F2E
:1027700026C081FF04C06091090184E005C082FF8A
:1027800007C06091090188E0689FB001112417C05B
:1027900090919D029923D1F060910801961788F7D6
:1027A0002091090188E0289F90011124929FA001A7
:1027B000939F500D112470E0CA010E94432B603892
:1027C000710540F46115710519F406C068E070E008
:1027D000862F08958FE7089581E0089580919E02E5
:1027E00080FF08C06091050170E07595679575954B
:1027F000679521C081FF06C06091050170E0759565
:10280000679519C082FF04C06091050170E010C097
:1028100090919C02992399F0609104019617A0F77A
:1028200080910501899FC001112470E00E94432B13
:102830006038710540F46115710519F406C061E056
:1028400070E0862F08958FE7089581E008958D3E0A
:1028500021F40E94AF13819504C08E3E29F40E949A
:10286000AF138093A20208958F3E21F40E94AF130C
:10287000819504C0803F29F40E94AF138093A10288
:102880000895893F19F40E94EE1305C08A3F31F480
:102890000E94EE1381958093A30208958B3F21F44B
:1028A0000E94EE13819504C08C3F29F40E94EE1320
:1028B0008093A40208959FE0980F983078F421E067
:1028C00030E0A90102C0440F551F9A95E2F7CA01F2
:1028D0009091A002892B8093A00208958D3F21F44E
:1028E00080919E0281600BC08E3F21F480919E02F8
:1028F000826005C08F3F29F480919E02846080939E
:102900009E0208958D3E39F49091A20297FF35C042
:102910001092A20259C08E3E29F49091A20219167B
:10292000BCF32BC09091A1028F3E29F497FF25C0E4
:102930001092A10249C0803F19F41916CCF31DC0B2
:102940009091A302893F29F41916BCF41092A302B6
:102950003BC08A3F19F497FF10C0F8CF8B3F39F482
:102960009091A40297FF09C01092A4022DC08C3F41
:1029700021F49091A4021916BCF39FE0980F9830AF
:1029800080F421E030E0A90102C0440F551F9A9560
:10299000E2F7CA0180959091A00289238093A0025A
:1029A00013C08D3F21F480919E028E7F0BC08E3F1D
:1029B00021F480919E028D7F05C08F3F29F4809184
:1029C0009E028B7F80939E028091A102811106C09E
:1029D0008091A202811102C010929D028091A302F7
:1029E000811106C08091A402811102C010929C0244
:1029F00008950E94BF232091A102211104C02091BB
:102A0000A202222321F090939B0280939A022091AC
:102A1000A302211104C02091A402222321F090934B
:102A20009902809398028FE992E00C942B22EF9206
:102A3000FF920F931F93CF93DF9300D000D000D06D
:102A4000CDB7DEB786E0EFE9F2E0DE011196019046
:102A50000D928A95E1F7E090A102F090A202009118
:102A6000A3021091A4021092A1021092A20210924D
:102A7000A3021092A402E11003C0FF2009F45DC07C
:102A800080919A0290919B020E94D723AC01909171
:102A90009D02992339F020910A0130E0241735076F
:102AA00058F04BC020910B018AE0289F900111241F
:102AB0002417350718F041C09F3F19F09F5F90938E
:102AC0009D02EE2061F00E94AF131E1414F09FEFE0
:102AD00001C091E0989F902D11249093A102FF20B6
:102AE00061F00E94AF131F1414F09FEF01C091E03A
:102AF000989F902D11249093A2023091A10233232C
:102B0000E1F02091A2022223C1F045EB3403C00181
:102B10001124992319F09093A10203C081E08093BE
:102B2000A10235EB2303C0011124992319F09093DE
:102B3000A20203C081E08093A202011103C011230D
:102B400009F45DC080919802909199020E94D72368
:102B5000AC0190919C02992339F02091060130E05C
:102B60002417350758F04BC0209107018AE0289FB1
:102B7000900111242417350718F041C09F3F19F028
:102B80009F5F90939C02002361F00E94EE13101649
:102B900014F09FEF01C091E0989F902D1124909325
:102BA000A302112361F00E94EE13111614F09FEF9F
:102BB00001C091E0989F902D11249093A402309130
:102BC000A3023323E1F02091A4022223C1F045EBBC
:102BD0003403C0011124992319F09093A30203C078
:102BE00081E08093A30235EB2303C00111249923D4
:102BF00019F09093A40203C081E08093A402809115
:102C0000A10281110BC08091A202811107C08091A5
:102C1000A302811103C08091A40281110E94F914C2
:102C2000EB82FC820D831E8386E0FE013196AFE9C4
:102C3000B2E001900D928A95E1F726960FB6F894CE
:102C4000DEBF0FBECDBFDF91CF911F910F91FF90DF
:102C5000EF900895EFE9F2E086E0DF011D928A959A
:102C6000E9F710929D0210929C0210929E02089524
:102C7000EF92FF920F931F93CF93DF938B01682FF7
:102C800011110AC0442329F0E82FF0E0E55EFC4F63
:102C90006491762F862F75C0212F30E0E82FF0E069
:102CA000442321F0E55EFC4FE491F0E046E0049F10
:102CB000C0011124CFEFD0E0BE010E942F2B4BEAC0
:102CC0004603C001479F900D1124800F911D800F76
:102CD000911D982F990F890FAE01421B530B4E9FE8
:102CE000D0014F9FB00D5E9FB00D11249B2F189FF8
:102CF000A0011124452F55278E01041B150B0E9F93
:102D0000A0010F9F500D1E9F500D11247E01E81A47
:102D1000F108E29E8001E39E100DF29E100D112439
:102D2000212F3327C21BD30BCE9F9001CF9F300D95
:102D3000DE9F300D112462307105A9F048F4611551
:102D4000710569F061307105C9F48B2F752F0DC0C5
:102D50006430710581F058F06630710579F47E2F8A
:102D60008B2F932F0DC0832F7B2F9E2F09C08E2F6B
:102D70007B2F952F05C08E2F732F02C07E2F852F9E
:102D8000692FDF91CF911F910F91FF90EF900895E0
:102D900041E00E943816089508950E94C8160895CB
:102DA000CF93DF93762FE901682F842F0E94CD16F1
:102DB000798368838A83DF91CF9108958091F802A7
:102DC000282F269530E02115310519F48170826095
:102DD00005C02532310524F0817088648093F802A3
:102DE000089588E090E00C94DE2BCF92DF92EF9272
:102DF000FF926B017C010E94DE16B701A60188E0FC
:102E000090E0FF90EF90DF90CF900C94FC2BE8EFD8
:102E1000F2E083E0808311828FEF828383831482C8
:102E200060817181828193810C94F5168091F80202
:102E300080FF02C08695089580E008959091FC027D
:102E4000933018F49F5F9093FC02882351F06091B7
:102E5000F8027091F9028091FA029091FB020C94B1
:102E6000F516089581E00C941E179091FC029923A9
:102E700019F091509093FC02882351F06091F80270
:102E80007091F9028091FA029091FB020C94F51670
:102E9000089581E00C94351770E00C94921F6091B6
:102EA00010018091F80280FF0AC080910F0123E099
:102EB000829FC001112483509D4F0C944C17809128
:102EC000110190911201891780F7E82FF0E09F011E
:102ED000220F331FE20FF31FE350FD4F11821082C8
:102EE00012828F5FF0CF9091F80290FF16C0909100
:102EF000110120911201921770F4E92FF0E0DF0127
:102F0000AA0FBB1FEA0FFB1FE350FD4F81836083B5
:102F100042839F5FF0CF0C944F170895CF93DF93B8
:102F200000D01F92CDB7DEB79091F80290FF0AC093
:102F30009E012F5F3F4F0E94D0164B8169818A818D
:102F40000E9473170F900F900F90DF91CF9108950B
:102F5000CF93DF93EC01EC81F0E0EA5EFD4F44910A
:102F6000E8EFF2E0628181810E948E178C818F5F91
:102F70008C83DF91CF910895CF93DF93EC01E8EF3D
:102F8000F2E0438162818C810E948E178C818F5F79
:102F90008C83DF91CF9108950F931F93CF93DF938D
:102FA00000D01F92CDB7DEB78C018091A5028111B0
:102FB0000AC09E012F5F3F4F4FEF6FEF0E94D01668
:102FC0008A818093A502F8018481813051F028F034
:102FD000823061F44091A5020AC08091A50240E0D0
:102FE00007C06091A50240E080E003C040E080E0BF
:102FF00060E00E947317F801848190E0019663E01D
:1030000070E00E94432B84830F900F900F90DF910C
:10301000CF911F910F910895AF92BF92CF92DF92FF
:10302000EF92FF920F931F93CF93DF9300D01F92E5
:10303000CDB7DEB7182FF62E042FE22E9091F802AE
:1030400090FF6DC0E92FE695AE2FB0E0AE55BE4FB4
:103050008C918093AF029E7F923061F49E012F5F2E
:103060003F4F812F0E94D0164B8169818A810E9437
:10307000731743C0823019F40091FB023EC08630C2
:1030800019F41091F90239C08930D9F38931A9F5C1
:10309000E9518E2F8170D82EE695F0E0EA5EFC4F64
:1030A000A590B490C12CBB2460911301C61618F5ED
:1030B0002C2D30E0A29EC001A39E900DB29E900DDB
:1030C000112470E00E942F2B812FD11002C0860F97
:1030D00001C0861B90911101290F311DA901440FD8
:1030E000551F240F351F23503D4F402F6F2D0E9439
:1030F000D016C394D9CF0E944F171093F902F092C3
:10310000FA020093FB02EE2051F06091F8027091F8
:10311000F9028091FA029091FB020E94F5160F903D
:103120000F900F90DF91CF911F910F91FF90EF9033
:10313000DF90CF90BF90AF900895E8EFF2E09181DB
:10314000282F4381628188E0890F0C940C1881E05C
:103150000C949D18E8EFF2E09181282F4381628161
:1031600088EF890F0C940C1881E00C94AA18E8EFF2
:10317000F2E0628128E0620F08F46FEF282F4381AC
:1031800081810C940C1881E00C94B718E8EFF2E000
:10319000628128E0621B08F460E0282F438181816E
:1031A0000C940C1881E00C94C618E8EFF2E043810F
:1031B00028E0420F08F44FEF282F628181810C94A0
:1031C0000C1881E00C94D518E8EFF2E0438128E078
:1031D000421B08F440E0282F628181810C940C1876
:1031E00081E00C94E41820E00C940C18FF920F93EB
:1031F0001F93CF93DF93EC01F12C0FEF10E0609160
:103200001301F616F0F4809111012F2D30E0280FF4
:10321000311DC901880F991F280F391F23503D4FB9
:1032200070E0C8010E94432B962F8C814091FB02D5
:103230006091FA02F99E800D11240E94D016F39439
:10324000DECF0E944F179A818C8190FF02C08F5F62
:1032500001C081508C83DF91CF911F910F91FF901E
:103260000895AF92BF92CF92DF92EF92FF920F93A9
:103270001F93CF93DF93FC01828180FF02C00FEF89
:1032800001C001E010E046E0A42E80911301181760
:1032900008F043C080911101C12ED12CE601C80F66
:1032A000D11DCE01880F991FC80FD91FC350DD4F04
:1032B000198218821A8234E0E32EF12CB12C80910D
:1032C000A7028B0D87302CF06A2D0E94212B892FAD
:1032D00005C087FF03C090911301890F082E000CD1
:1032E000990BC816D90691F48091FB028E9DA0011E
:1032F0008F9D500D112455954795559547959E01E5
:103300006091FA028091F9020E94D016B00EF1E0AD
:10331000EF1AF108A1F61F5FB8CF0E944F178091F6
:10332000A702013031F4811102C080911301815054
:1033300007C090E001966091130170E00E94432B5A
:103340008093A702DF91CF911F910F91FF90EF9093
:10335000DF90CF90BF90AF900895CF9380911101EF
:1033600090911201891770F4E82FF0E09F01220F6D
:10337000331FE20FF31FE350FD4F118210821282C0
:103380008F5FF0CFC0E060911301C617C0F5EC2F3E
:10339000F0E070E0CF010E94432B20911101820FD9
:1033A0002091A602022E000C330B90E0E217F307E7
:1033B000CCF020910E01022E000C330B2E173F078C
:1033C0008CF09C01220F331F820F931F9C0123500E
:1033D0003D4F4091FB026091FA028091F9020E94F8
:1033E000D0160BC0FC01EE0FFF1F8E0F9F1FFC01BC
:1033F000E350FD4F118210821282CF5FC4CF0E9432
:103400004F1720910D018091A602820F8093A60292
:1034100090910E01920F90930E0119165CF4082EF4
:10342000000C990B4091130150E041505109841751
:1034300095071CF0219520930D01CF9108958F924F
:103440009F92AF92BF92CF92DF92EF92FF920F9333
:103450001F93CF93DF938C01FC014481C42FD0E0F4
:103460009E01DE010E94872B9B01AC010E949D2BD7
:103470006B017C01E0E2F0E0EC1BFD0BA5E5B0E0A8
:103480009B01AC010E949D2B4B015C019F01DF0160
:103490000E947F2B9B01AC010E94A82B9B01AC01D9
:1034A0002C0D3D1D4E1D5F1DC501B4010E94572B03
:1034B000C22FD22F2A3228F4F3E02F9F900111243B
:1034C0000DC025E530E02C1B3109C901880F991F7B
:1034D000280F391F37FF02C02F5F3F4F35952795C3
:1034E000C22FC095F12C85E5E82EED1A80911301CD
:1034F000F816C8F4F1FC02C08E2D01C08D2F9091FA
:1035000011012F2D30E0290F311DA901440F551F46
:10351000240F351F23503D4F4C2F6091FA020E941B
:10352000D016F394E3CF0E944F17F80184818111E4
:1035300002C091E003C0803219F49FEF90930C0118
:1035400090910C01890FF8018483DF91CF911F9135
:103550000F91FF90EF90DF90CF90BF90AF909F9032
:103560008F9008950F931F93CF93DF93EC0100E0AA
:1035700010E080911301282F30E00217130724F583
:10358000909111019801290F311DA901440F551F78
:10359000240F351F23503D4F869590E04C8108172E
:1035A00019071CF4442331F002C0411103C04091BB
:1035B000FB0201C040E06091FA028091F9020E9492
:1035C000D0160F5F1F4FD5CF0E944F178C8190E010
:1035D0000196817099278C83DF91CF911F910F9174
:1035E0000895E8EFF2E080818E7F808360817181B1
:1035F000828193810E94F5161092B0022FEF80E72E
:1036000092E0215080409040E1F700C000000C940F
:103610004F176091F802669570E04BE050E084E14E
:1036200091E00E94BC2B892B19F481E08093B002B9
:103630000E94BF239093A9028093A80208959091BD
:10364000F80290FF35C09170811102C0926006C0EF
:10365000853210F0986402C0880F982B9093F8027E
:10366000662351F06091F8027091F9028091FA029C
:103670009091FB020E94F5166091F802669570E049
:103680004BE050E084E191E00E94BC2B892B19F0C3
:103690001092B00202C00E94091B81E08093AB022D
:1036A0004091FB026091FA028091F9020C94F318A8
:1036B0000895682F9091F802969581E0890F8532E0
:1036C00008F081E00C941F1B81E00C94591B682FBB
:1036D0009091F80296958FEF890F09F484E20C948B
:1036E0001F1B81E00C94671B61E00C941F1BE8EF2B
:1036F000F2E080818160808386950C94741B8091B8
:10370000F80280FD0C94F11A0C94771B60E00C9485
:103710001F1B8091AE0281112EC00E945C0E811190
:1037200004C00E94040F0E9407170E94F1166093C4
:10373000F8027093F9028093FA029093FB026E7F75
:1037400061F40E9407170E94F1166093F8027093CB
:10375000F9028093FA029093FB020E94DE16109207
:10376000B0028091F80280FF03C086950E94861BFC
:1037700081E08093AE0208950F931F93CF93DF9360
:103780008091B002882309F485C08091AF02E09156
:10379000F802E695E81BE093AA02823049F4F0E0D3
:1037A000EE5EFD4FE491CE2FD0E008EA17E149C06C
:1037B000863049F4F0E0E15FFD4FE491CE2FD0E098
:1037C0000CEB17E13EC0893051F4E695F0E0E45F80
:1037D000FD4FE491CE2FD0E006EF18E132C08F30DC
:1037E00051F4E695F0E0E75FFD4FE491CE2FD0E095
:1037F00001E319E126C0853149F4F0E0EA5FFD4FAD
:10380000E491CE2FD0E00DEA19E11BC0883181F0A0
:10381000833239F4E4E0F2E0C591D4910CEC17E185
:1038200010C0843251F4C4EFD1E002EB1AE109C0B8
:10383000C8E2D0E00FE11AE104C0C0EDD7E00CEC23
:1038400016E18091AB02882361F01092AB020E94D6
:10385000BF239093A9028093A8021092AD02109208
:10386000AC020E94BF23E091A802F091A9028E1B36
:103870009F0B8F3F9F4770F4EC0FFD1FF093A90241
:10388000E093A80288EA92E0F801DF91CF911F91BE
:103890000F910994DF91CF911F910F910895882383
:1038A00011F0FA0101C0FB010994CF93DF93C82FF7
:1038B000D62F0E9416178C1740F00E9416178D17EE
:1038C00020F4DF91CF910C94641B8C2FDF91CF916A
:1038D0000C94741B1F93CF93DF93FB011281111182
:1038E000C3C0EC010E94730D8272CD3CFCE5DF0782
:1038F00009F49AC0A8F5C73CECE5DE0709F476C0E8
:10390000A8F4C43C9CE5D90709F45FC028F4C33C83
:10391000DC4509F457C054C0C53C9CE5D90709F4FF
:1039200059C0C63CDC4509F45CC04AC0CA3CFCE551
:10393000DF0709F46AC050F4C83CECE5DE0709F47F
:103940005AC0C93CDC4509F45BC03AC0CB3C9CE59D
:10395000D90709F45FC0CC3CDC4509F460C030C035
:10396000C23DFCE5DF0709F46FC088F4CF3C9CE55D
:10397000D90709F460C008F45CC0C03DFCE5DF076E
:1039800009F45CC0C13DDC4509F45BC019C0C53D0C
:103990009CE5D90709F460C050F4C33DFCE5DF079E
:1039A00009F455C0C43DDC4509F454C009C0C63D06
:1039B0009CE5D90709F455C0CE35DD4509F454C05E
:1039C00011E052C00E947F1B4FC041E75BE164E6FB
:1039D0007BE104C044E65BE161E77BE10E944F1CB0
:1039E00043C044EB58E167EA78E1F8CF47EA58E191
:1039F00064EB78E1F3CF42ED58E163EC78E1EECF90
:103A000043EC58E162ED78E1E9CF40EF58E161EE37
:103A100078E1E4CF41EE58E160EF78E1DFCF49E4AF
:103A200057E162E377E1DACF42E357E169E477E116
:103A3000D5CF81E017C065E082E010C068E086E085
:103A40000DC06EE089E00AC064E18FE007C067E165
:103A500085E104C088E106C062E289E10E94551C4C
:103A600003C083E20E94741B812FDF91CF911F91CD
:103A7000089586E090E00C94D62B682F86E090E0C5
:103A80000C94EA2B80910F038470896180930F035B
:103A90000C943D1D0E945C0E811104C00E94040F15
:103AA0000E94421D0E94391D80930F03282F2695E6
:103AB0002695269530E02430310524F08770886102
:103AC00080930F0380910F0380FF04C08695869535
:103AD000869501C080E00C94B61E20910F03822FC2
:103AE000869586958695482F50E04330510554F4CD
:103AF0008F5F982F990F990F990F822F8770892BBD
:103B000080930F0380910F03816080930F030E94C5
:103B10003D1D80910F038695869586950C94B61E63
:103B200080910F03982F969596959695A1F0915EAA
:103B3000990F990F990F8770892B80930F03887FB6
:103B400091E009F490E080910F0390FB80F980935D
:103B50000F030E943D1D80910F03869586958695E3
:103B60000C94B61E80910F0380FD13C0816080937A
:103B70000F03813019F489E080930F0380910F03C4
:103B80000E943D1D80910F038695869586950C9425
:103B9000B61E089580910F0380FF08C08E7F80932A
:103BA0000F030E943D1D80E00C94B61E0895809185
:103BB0000F0380FD0C94CA1D0C94B21D90910F034D
:103BC000892F8695869586958F5F8F719770843043
:103BD00038F4880F880F880F892B80930F0302C059
:103BE00090930F0380910F03887F91E009F490E098
:103BF00080910F0390FB80F980930F030E943D1D7D
:103C000080910F038695869586950C94B61E843018
:103C100008F083E090910F039770282F220F220F56
:103C2000220F922B90930F03987F21E009F420E05C
:103C300090910F0320FB90F990930F030C94B61E04
:103C40000E94071E80910F030C943D1D9C01FB01F7
:103C50008281882349F12E3BFCE53F07C9F040F4FF
:103C60002C3BECE53E0769F02D3B3C4561F00895A7
:103C7000203C9CE5390791F070F0213C3C4589F0EF
:103C8000089583E001C080E00E94201E80E0089536
:103C90000E94901DFBCF0E946D1DF8CF0E94D71D82
:103CA000F5CF0E94DE1DF2CF81E00895809A8898BA
:103CB0000895889A0895889808951F920F920FB6D4
:103CC0000F9211242F933F934F935F936F937F93A2
:103CD0008F939F93AF93BF93EF93FF930E945B1ECD
:103CE000FF91EF91BF91AF919F918F917F916F91D4
:103CF0005F914F913F912F910F900FBE0F901F90AA
:103D000018951F920F920FB60F9211242F933F9385
:103D10004F935F936F937F938F939F93AF93BF93D3
:103D2000EF93FF9320918800309189008091860065
:103D3000909187006AEF70E00E942F2B6B5F7F4F9E
:103D40006217730710F40E94591EFF91EF91BF9103
:103D5000AF919F918F917F916F915F914F913F9123
:103D60002F910F900FBE0F901F9018958F929F92DA
:103D7000AF92BF92CF92DF92EF92FF920F931F9379
:103D8000CF93DF93C82F8430A8F4811114C08091A1
:103D9000880090918900892B51F080916F008D7F70
:103DA00080936F0080916F008E7F80936F000E94E0
:103DB0005B1E11C0C3E08091880090918900892B1F
:103DC00051F480916F00826080936F0080916F004A
:103DD000816080936F00A0918600B09187002C2FA6
:103DE00030E00E94872B23E030E040E050E00E946A
:103DF000572B0027122F232F342F012F122F232F61
:103E0000332780918600909187006CE070E00E94DB
:103E10002F2B6017710730F0C80169E070E00E9435
:103E20002F2B5EC08091860090918700E0908600E5
:103E3000F0908700E0918600F0918700C6E0D0E026
:103E4000BE010E942F2B060F171F211D311D480197
:103E5000590185E0880C991CAA1CBB1C8A95D1F7D6
:103E6000C701BE010E942F2B6F01E12CF12CA7018D
:103E70009601260F371F411D511DC501B4010E9437
:103E8000572B69017A01E0918600F0918700CA0101
:103E9000B9010E94112B9B01AC01DF010E949D2BF7
:103EA0009B01AC01C701B6010E94112BDC01CB01C3
:103EB0002FE0B695A795979587952A95D1F700910C
:103EC00086001091870020E030E0081719072A07C4
:103ED0003B0728F46091860070918700CB01BC01FC
:103EE0007093890060938800DF91CF911F910F91AB
:103EF000FF90EF90DF90CF90BF90AF909F908F900A
:103F0000089508950E94561E82E08093800089E102
:103F1000809381008FEF9FEF9093870080938600BE
:103F20000C944A1D219A25B12D7F35B132604FB7CF
:103F3000F894FC01CB01880F991F680F791F6E0F51
:103F40007F1FE617F70789F0819198E035B90000E7
:103F500000C087FF25B9880F000000C000C000C066
:103F600025B900C09A9591F7ECCF4FBF8FE594E04B
:103F70000197F1F700C000000895CF93DF93EC01A3
:103F8000FB018281882309F43CC1C430FDE5DF07D1
:103F900060F4CB3F9CE5D90788F49E0122503C4554
:103FA0002431310508F02EC109C0C236EDE5DE0727
:103FB00029F0C63AFDE5DF0709F024C10E946F0E23
:103FC0009093E3028093E202C1318CE5D80709F4B3
:103FD000C6C008F042C0C930ECE5DE0709F49BC05A
:103FE00000F5C5308CE5D80709F485C078F4C330F6
:103FF000ECE5DE0709F478C008F07AC0C230DC4591
:1040000009F0F5C08091E2028160EFC0C7309CE505
:10401000D90709F478C008F07AC08091E202806183
:10402000E4C0CD30FCE5DF0709F487C058F4CB309D
:104030009CE5D90709F479C008F07BC08091E202C1
:1040400088606FC0CF30FCE5DF0709F480C008F05E
:1040500082C08091E202877FC8C0CE3F9CE5D9072D
:1040600009F471C000F5C531FCE5DF0709F485C02E
:1040700068F4C3319CE5D90709F475C008F095C010
:104080000E9420088091E2028F77AFC0CC3FFCE510
:10409000DF07A9F108F054C0CB3FDC4509F0A7C009
:1040A0008091E30240C0C230EDE5DE0709F489C02B
:1040B00058F4C1158DE5D80709F45AC008F069C055
:1040C0008091E30282602FC0C236EDE5DE0709F47D
:1040D0007CC0C63AFDE5DF0709F481C0C330DD4589
:1040E00009F085C080E06EC08091E20282607DC0F0
:1040F0008091E20216C08091E202886076C08091D1
:10410000E30282604FC08091E20280626EC08091C3
:10411000E20280646AC00E9420088091E202806806
:1041200064C0846062C081603DC08091E2028E7F85
:104130005CC08091E2028D7F58C08091E20216C07F
:104140008091E30218C08091E3028D7F2BC08091A3
:10415000E2028F7E4AC08091E2028F7D46C080914C
:10416000E2028F7B42C08091E202877F8B7F3DC05D
:104170008091E3028D7F8E7F15C08091E20282FBE9
:10418000222720F991E0922790FB82F990FB83F996
:104190002CC08091E302982F909591708E7F892B8F
:1041A00090FB81F98093E30222C00E942008809155
:1041B000E20287FB222720F991E0922790FB87F902
:1041C00014C081E00E94060F12C08091E20284FBBD
:1041D000222720F991E0922790FB84F906C0809174
:1041E000E202982F909590FB80F98093E2028091F3
:1041F000E2029091E3020E94800E0E94200880E07B
:1042000001C081E0DF91CF910895CF93DF93863194
:104210009C4541F5EB010E94730D982F8A812091F6
:10422000020130910301882379F09A7A81E009F440
:1042300080E08093B102911102C069E201C065E3A0
:10424000C9010E94FB220AC08091B102811102C003
:1042500069E201C065E3C9010E9406230E94B50D11
:1042600080E001C081E0DF91CF9108950F931F930B
:10427000CF93DF93C42FD22FFC0182818823C9F012
:104280004093B4020E94BF239093B3028093B20282
:1042900080E28C0F883008F057C0C77081E001C001
:1042A000880FCA95EAF7DF91CF911F910F910C9477
:1042B0007D058091B402481330C08091B202909184
:1042C000B3020E94D723883C910538F510E21D0FF8
:1042D000CD17B9F080E28C0F883040F4C77081E0D0
:1042E00001C0880FCA95EAF70E948405183028F5A6
:1042F00081E09D2F977001C0880F9A95EAF70E9480
:104300007D05802F0E9474051830F0F4D77081E08D
:1043100001C0880FDA95EAF70AC080E28C0F883076
:1043200098F4C77081E001C0880FCA95EAF7DF9161
:10433000CF911F910F910C948405802FDF91CF9125
:104340001F910F910C947405DF91CF911F910F91E4
:1043500008950F939C01CB01243F4CE5340731F1C4
:1043600088F4293DFCE53F07D9F02A3D4CE53407A8
:1043700079F1283D3C45A9F506E221EE41EE68EDD4
:104380007CE52BC0263FFCE53F07E1F0A8F0273F86
:104390003C4539F507E225EE46EE67EF7CE51DC0AA
:1043A00007E225EE45EE69ED7CE517C006E221EE59
:1043B00040EE64EF7CE511C007E225EE44EE65EFC8
:1043C0007CE50BC006E221EE42EE66EF7CE505C01F
:1043D00008E221E045EE6AED7CE50E94362180E0AE
:1043E00008C0FC018281882319F01092B40201C038
:1043F00081E00F9108959093C9018093C8010895B9
:104400009093BA028093B9020895E091B902F091B5
:10441000BA02309721F00190F081E02D099480E0FC
:104420000895E091B902F091BA02309799F0209185
:104430002B01222359F02091E20227FF07C0DC0163
:104440002C9111962C93119726E02C930280F381E6
:10445000E02D09940895E091B902F091BA023097E5
:1044600039F022E0DC012C930480F581E02D0994E1
:1044700008952091B7023091B8022817390771F0DA
:104480009093B8028093B702E091B902F091BA021A
:10449000309721F00680F781E02D0994089520914E
:1044A000B5023091B6022817390771F09093B60221
:1044B0008093B502E091B902F091BA02309721F0F1
:1044C0000084F185E02D09940895FC0132968091D5
:1044D0002B01882331F08091E20287FF02C09EE128
:1044E00001C096E080E0915028F021912223D9F379
:1044F0008F5FF9CF0895662351F120912B0122237C
:10450000E9F02091E20227FF19C0462F4695469513
:1045100046954E31E0F4677021E030E002C0220F92
:10452000331F6A95E2F7FC01E40FF11D828190E0F0
:104530002823392381E0232B69F409C0FC0132963A
:1045400008962191621729F0E817F907D1F780E062
:10455000089581E008959C01FC0132969FEF80E070
:104560004191461789F09F3F19F4411101C0982FDE
:104570008F5F8630A9F79F3F39F0F901E90FF11DF0
:1045800097FDFA956283089508959C012A5F3F4F35
:10459000FC014281461301C01282019682179307E3
:1045A000B9F70895262F2695269526952E3168F47D
:1045B000FC01E20FF11D677021E030E001C0220F25
:1045C0006A95EAF78281282B22830895262F269563
:1045D000269526952E3170F4FC01E20FF11D6770CF
:1045E00021E030E001C0220F6A95EAF72095828130
:1045F00028232283089520912B01222329F0209142
:10460000E20227FD0C94D2220C94AB2220912B01C4
:10461000222329F02091E20227FD0C94E6220C943B
:10462000C52220912B01FC013296222331F080918A
:10463000E20287FF02C08EE101C086E0DF011D9229
:104640008A95E9F7089508950C94232383E08093D5
:10465000BB020C942423811102C081E001C082E0DE
:104660008093BB020C9424230C942B2381E0809331
:10467000BB020C9424230C94362308950C943D2300
:104680000C943E230C943D230C943D230C943D2329
:10469000CF930E9444230E9410130E944223C0E043
:1046A0008C2F0E943A12892B29F4CF5FC530C1F7B5
:1046B00080E001C081E0CF91089508951F920F928C
:1046C0000FB60F9211248F939F93AF93BF93809156
:1046D000BC02811113C08091100390911103A0912D
:1046E0001203B09113034196A11DB11D80931003D5
:1046F00090931103A0931203B0931303BF91AF9152
:104700009F918F910F900FBE0F901F9018958091E1
:104710001803843031F10E94BE031092BC0220E4E1
:1047200088E190E00FB6F894A895809360000FBEE2
:104730002093600083B7817F846083BF83B78160EB
:1047400083BF7894889583B78E7F83BF0FB6F89424
:10475000A89580916000886180936000109260004D
:104760000FBE08950E9420080C94C50382E084BD0A
:1047700093E095BD9AEF97BD80936E0008952FB793
:10478000F8948091100390911103A0911203B091BD
:1047900013032FBF08952FB7F89460911003709101
:1047A000110380911203909113032FBF08959C0170
:1047B0004FB7F8948091100390911103A0911203C8
:1047C000B09113034FBF821B930B089578941F92EF
:1047D0000F920FB60F9211248F939F93AF93BF93B5
:1047E0008091100390911103A0911203B0911303D3
:1047F0000196A11DB11D8093100390931103A09306
:104800001203B0931303BF91AF919F918F910F90BB
:104810000FBE0F901F90189581E08093E00080E21A
:104820008093D8001092C9008FE19EE40197F1F7C0
:1048300000C0000087E090EBDC018093210390939F
:104840002203A0932303B09324039CE088E10FB6D6
:10485000F894A895809360000FBE90936000FFCFFE
:104860008091E0020895089522E02093E9002FEF5F
:104870003091E800215035FD06C035ED3A95F1F74D
:1048800000002111F5CF2091E80025FF0BC040E08A
:1048900050E066E070E00E9473268091E8008E7719
:1048A0008093E8000895CF93DF9320912B0122237A
:1048B00039F02091E20227FF03C060E222E002C04B
:1048C00068E021E02093E9002FEF3091E8002150CB
:1048D00035FD06C035ED3A95F1F700002111F5CF11
:1048E0002091E80025FF1DC0EC0180912B01811172
:1048F00005C040E050E068E070E003C070E040E0D8
:1049000050E0CE010E9473268091E8008E7780935C
:10491000E80080E2FE01A0ECB2E001900D928A95E1
:10492000E1F7DF91CF9108958093BD027093BF02AC
:104930006093BE0280911803843001F582E0809379
:10494000E9008FEF9091E800815095FD06C095ED4C
:104950009A95F1F700008111F5CF8091E80085FF6D
:104960000DC040E050E063E070E08DEB92E00E940B
:1049700073268091E8008E778093E8000895BC014B
:1049800084E00C949424BC0183E00C9494248091E2
:104990001703811109C00E9404280E946128809198
:1049A000E20084608093E200089510921703089556
:1049B0000C943B236091140381E0611101C080E0FD
:1049C0000C9426239091180381E0943009F080E044
:1049D000609114030C942B2342E061EC81E00E946F
:1049E0007D2742E261EC82E00E947D2790911803CE
:1049F00081E0943009F080E0609114030C9434233A
:104A000080911A03833009F461C030F4813071F071
:104A1000823009F49AC008958A3009F486C08B3038
:104A200009F46CC0893009F0A8C020C08091190336
:104A3000813A09F0A2C08091E800877F8093E80066
:104A400080911D0390911E03892B21F460E280EC7C
:104A500092E003C060E080E090E070E00E94BE263B
:104A60008091E8008B778093E80008958091190386
:104A7000813209F082C080911D0390911E0302973C
:104A800008F07BC08091E800877F8093E8008091E8
:104A9000E80082FD05C0809118038111F8CF6DC038
:104AA0002091F3008091F20090E0922B029731F474
:104AB0008091F100813011F0863021F48091F10075
:104AC0008093E0028091E8008B7753C080911903B6
:104AD000813A09F052C080911D0390911E03892BE9
:104AE00009F04BC08091E800877F8093E8008091B7
:104AF000E80080FFFCCF80912B0136C08091190324
:104B00008132D9F580911D0390911E03892BA9F55F
:104B10008091E800877F8093E8000E94B22780910F
:104B20001B0380932B010C94200880911903813280
:104B300021F58091E800877F8093E8000E94B227EA
:104B400080911C038093E102089580911903813ABA
:104B5000A1F48091E800877F8093E8008091E800CD
:104B600080FFFCCF8091E1028093F1008091E8000A
:104B70008E778093E8000C94B227089584B7877FDE
:104B800084BF0FB6F894A8958091600088618093E7
:104B90006000109260000FBE90E080E80FB6F894BD
:104BA00080936100909361000FBE0C9436230E94A5
:104BB00004280E946128E2EEF0E080818460808316
:104BC00078940C94F62A8FE191E00C940022809165
:104BD00018038530A9F480911803853079F40E9478
:104BE0008723809116038823B1F30E9448238823EA
:104BF00091F30E945D260E942008EDCF0C94B22311
:104C0000089508950C940426292F33272330310565
:104C1000C9F060F42130310581F02230310509F00E
:104C200044C08BE390E029E334E043C021323105F6
:104C3000E1F02232310549F138C082E190E024E709
:104C400034E037C099278130910549F028F0029768
:104C500061F5EBE1F4E005C0E5E3F4E002C0E7E272
:104C6000F4E0849190E09F0124C06115710541F04A
:104C700061307105D1F489E090E024E634E019C098
:104C800089E090E02BE434E014C06115710541F037
:104C90006130710551F486EB90E026E834E009C0FC
:104CA00080E490E02CE335E004C080E090E020E078
:104CB00030E0FA0131832083089580E189BD82E1EB
:104CC00089BD09B400FEFDCF8091D8008F7D80930F
:104CD000D8008091E00082608093E0008091E00045
:104CE00081FDFCCF0895CF92DF92EF92FF920F9358
:104CF0001F93CF93DF93EC018B017A010E94D127A0
:104D0000811133C0E114F10439F0F7018081918100
:104D1000081B190BC80FD91FC12CD12C0115110567
:104D200019F18091E80085FD16C08091E8008E772A
:104D30008093E800E114F10449F0F701808191814A
:104D4000C80ED91ED182C08285E00FC00E94D12733
:104D5000882321F30AC089918093F1000150110941
:104D6000FFEFCF1ADF0ADACF80E0DF91CF911F91FA
:104D70000F91FF90EF90DF90CF90089520911F0347
:104D8000309120032617370748F06115710539F473
:104D90002091E8002E772093E80001C0B901FC01C2
:104DA00020E06115710579F1809118038823F1F1F4
:104DB0008530F1F18091E80083FD3CC08091E800EE
:104DC00082FD2EC08091E80080FFEBCF2091F300A0
:104DD0008091F20090E0922B6115710551F08830BE
:104DE000910538F421912093F100615071090196E9
:104DF000F3CF21E0089709F020E08091E8008E775A
:104E00008093E800CECF2111CFCF0AC08091180344
:104E1000882361F0853061F08091E80083FD0AC04D
:104E20008091E80082FFF2CF80E0089582E008954B
:104E300083E0089581E0089520911F0330912003BD
:104E40002617370748F06115710539F42091E800FD
:104E50002E772093E80001C0B901FC0120E0611524
:104E6000710591F180911803882309F440C08530C1
:104E700009F43FC08091E80083FD3DC08091E800C7
:104E800082FD2FC08091E80080FFE9CF2091F300E0
:104E90008091F20090E0922B6115710559F08830F5
:104EA000910540F424912093F100319661507109ED
:104EB0000196F2CF21E0089709F020E08091E80008
:104EC0008E778093E800CBCF2111CCCF0AC08091A0
:104ED0001803882361F0853061F08091E80083FD3C
:104EE0000AC08091E80082FFF2CF80E0089582E05E
:104EF000089583E0089581E00895982F973068F52C
:104F00009093E900981739F07091EC002091ED0032
:104F10005091F00003C0242F762F50E021FD02C0F5
:104F20009F5FECCF3091EB003E7F3093EB003091F0
:104F3000ED003D7F3093ED003091EB003160309318
:104F4000EB007093EC002093ED005093F000209163
:104F5000EE0027FDE5CF80E008958F708093E90093
:104F600081E008958091190387FF11C08091E800C6
:104F700082FD05C0809118038111F8CF11C0809186
:104F8000E8008B770BC080911803882349F080914B
:104F9000E80080FFF8CF8091E8008E778093E800EA
:104FA00008952091E4003091E50095E64091EC00F1
:104FB000842F817040FF23C08091E80080FD1DC0D8
:104FC00080911803882399F0853099F08091EB0047
:104FD00085FD11C04091E4005091E500241735078C
:104FE00029F3915011F09A01E1CF84E0089582E015
:104FF000089583E0089581E0089580E00895409148
:10500000E80042FFDDCF08950E9472280E947A28AE
:10501000E0EEF0E0808181608083E8EDF0E0808167
:105020008F77808319BCA7EDB0E08C918E7F8C9335
:1050300080818F7E80831092170308950F931F93B2
:10504000CF93DF930E9472280E947A28C8EDD0E0A7
:1050500088818F77888388818068888388818F7D25
:10506000888319BC1092180310921403109216032F
:105070001092150300EE10E0F80180818B7F808391
:1050800088818160888342E060E080E00E947D2723
:10509000E1EEF0E080818E7F8083E2EEF0E08081BF
:1050A00081608083808188608083F80180818E7F29
:1050B0008083888180618883DF91CF911F910F91D8
:1050C0000895E8EDF0E080818F7E8083E7EDF0E0E9
:1050D00080818160808384E082BF81E080931703B8
:1050E0000C941E28E8EDF0E080818E7F8083109282
:1050F000E20008951092DA001092E10008951F92E4
:105100000F920FB60F9211242F933F934F935F93FB
:105110006F937F938F939F93AF93BF93EF93FF937F
:105120008091E10082FF0BC08091E20082FF07C006
:105130008091E1008B7F8093E1000E94F52A8091AD
:10514000DA0080FF1FC08091D80080FF1BC08091D3
:10515000DA008E7F8093DA008091D90080FF0DC045
:1051600080E189BD82E189BD09B400FEFDCF81E007
:10517000809318030E94C72405C019BC109218031D
:105180000E94D5248091E10080FF19C08091E20047
:1051900080FF15C08091E2008E7F8093E2008091B5
:1051A000E20080618093E2008091D8008062809369
:1051B000D80019BC85E0809318030E94DA248091FE
:1051C000E10084FF30C08091E20084FF2CC080E1C8
:1051D00089BD82E189BD09B400FEFDCF8091D80070
:1051E0008F7D8093D8008091E1008F7E8093E100D5
:1051F0008091E2008F7E8093E2008091E2008160E6
:105200008093E20080911403882311F084E007C0AA
:105210008091E30087FD02C081E001C083E08093BC
:1052200018030E94E2248091E10083FF29C080914D
:10523000E20083FF25C08091E100877F8093E10039
:1052400082E080931803109214038091E1008E7F16
:105250008093E1008091E2008E7F8093E200809154
:10526000E20080618093E20042E060E080E00E9422
:105270007D278091F00088608093F0000E94D82400
:10528000FF91EF91BF91AF919F918F917F916F911E
:105290005F914F913F912F910F900FBE0F901F90F4
:1052A00018951F920F920FB60F9211242F933F93D0
:1052B0004F935F936F937F938F939F93AF93BF931E
:1052C000CF93DF93EF93FF93C091E900CF7080916C
:1052D000EC00D82FD17080FDD0E81092E9008091C9
:1052E000F000877F8093F00078940E9495291092B7
:1052F000E9008091F00088608093F000CD2BCF70A2
:10530000C093E900FF91EF91DF91CF91BF91AF91F1
:105310009F918F917F916F915F914F913F912F91CD
:105320000F900FBE0F901F9018951F93CF93DF9390
:10533000CDB7DEB7AA970FB6F894DEBF0FBECDBFCC
:10534000E9E1F3E08091F100819323E0E132F2079B
:10535000C9F70E9400258091E80083FF2EC180914B
:10536000190390911A03492F50E04A30510508F073
:1053700024C1FA01EE59FF4F0C94792B803821F0AB
:10538000823809F01AC108C0809115039091160364
:10539000992389F082600FC080911D038F70873040
:1053A00008F00BC18093E9008091EB0085FB882712
:1053B00080F91092E9009091E800977F9093E800BF
:1053C0008093F1001092F100D1C0282F2D7F09F0B9
:1053D000F4C0882319F0823061F0EFC080911B0384
:1053E000813009F0EAC0933009F080E08093160321
:1053F0002EC080911B0381112AC080911D038F70E4
:105400002FEF280F263008F0D8C08093E9002091B4
:10541000EB0020FF1CC0933021F48091EB008062F0
:1054200014C09091EB0090619093EB0021E030E08C
:10543000A90102C0440F551F8A95E2F74093EA0084
:105440001092EA008091EB0088608093EB0010924C
:10545000E9008091E800877F8093E8000E94B227EE
:10546000ACC08111AAC010911B031F778091E3008B
:105470008078812B8093E3008091E800877F809380
:10548000E8000E94B2278091E80080FFFCCF809165
:10549000E30080688093E300111102C082E001C044
:1054A00083E08093180389C08058823008F085C05B
:1054B00080911B0390911C038C3D53E0950779F577
:1054C00083E08A838AE289834FB7F894DE011396DA
:1054D00020E03EE051E2E32FF0E050935700E491EA
:1054E00020FF03C0E295EF703F5FEF708E2F90E0DA
:1054F000EA3010F0C79601C0C0968D939D932F5F40
:10550000243149F74FBF8091E800877F8093E800FE
:105510006AE270E0CE0101960E94BE2616C060913C
:105520001D0370911E03AE014F5F5F4F0E94022664
:10553000BC01892B09F441C09091E800977F9093BA
:10554000E80089819A810E941C278091E8008B776E
:105550008093E80032C0803881F58091E800877F31
:105560008093E800809114038093F1008091E8001B
:105570008E7772CF811121C080911B0390911C0303
:1055800099270297D4F48091E800877F8093E80000
:1055900080911B03809314030E94B227809114030F
:1055A000811106C08091E30087FD02C081E001C047
:1055B00084E0809318030E94EC248091E80083FF2C
:1055C0000AC08091E800877F8093E8008091EB001B
:1055D00080628093EB00AA960FB6F894DEBF0FBEF0
:1055E000CDBFDF91CF911F9108950895CF93809102
:1055F00018038823A1F0C091E900CF709091EC00CE
:10560000892F817090FD80E8C82B1092E90080916D
:10561000E80083FD0E949529CF70C093E900CF91E7
:105620000895DB018F939F930E949D2BBF91AF91B3
:10563000A29F800D911DA39F900DB29F900D1124EC
:10564000089587FB082E062687FD819567FD6195E5
:105650000E94B02B0EF4919507FC81950895AA1B2A
:10566000BB1B51E107C0AA1FBB1FA617B70710F04D
:10567000A61BB70B881F991F5A95A9F7809590957F
:10568000BC01CD01089597FB072E16F4009407D0B6
:1056900077FD09D00E942F2B07FC05D03EF4909592
:1056A00081959F4F0895709561957F4F0895A1E270
:1056B0001A2EAA1BBB1BFD010DC0AA1FBB1FEE1F8C
:1056C000FF1FA217B307E407F50720F0A21BB30BD7
:1056D000E40BF50B661F771F881F991F1A9469F753
:1056E00060957095809590959B01AC01BD01CF01AF
:1056F0000895EE0FFF1F0590F491E02D09940E948C
:10570000872B332312F48A1B9B0B0C94982BA29F9C
:10571000B001B39FC001A39F700D811D1124911D85
:10572000B29F700D811D1124911D08950E94872B39
:10573000B7FF0895821B930B08950E94872BA59FA6
:10574000900DB49F900DA49F800D911D112408957C
:10575000B7FF0C949D2B0E949D2B821B930B0895E9
:10576000991B79E004C0991F961708F0961B881FB3
:105770007A95C9F780950895FC014150504030F06A
:1057800001900616D1F73197CF0108958827992700
:105790000895FB01DC0104C08D910190801921F472
:1057A00041505040C8F7881B990B0895F999FECFD6
:1057B00092BD81BDF89A992780B50895A6E1B0E021
:1057C00044E050E00C94102CA8E1B0E042E050E03E
:1057D0000C94102C262FF999FECF92BD81BDF89A1A
:1057E000019700B4021639F01FBA20BD0FB6F89425
:1057F000FA9AF99A0FBE08950396272F0E94EB2B71
:105800000E94EA2B252F0E94EB2B242F0C94EB2BCC
:105810000196272F0E94EB2B0C94EA2BDC01CB0185
:10582000FC01F999FECF06C0F2BDE1BDF89A3196B0
:1058300000B40D9241505040B8F70895F894FFCF4E
:10584000C8006002280850011E0A1401010102006C
:105850000600060601191A1B1C1D1E1F20212230DE
:105860002453243424C324BF24332401E200E90058
:10587000EA00B500B600B700CD008301CC008A0174
:10588000920194012102230224022502260227020A
:105890002A02B300B4006F007000818283E200E945
:1058A00000EA00B500B600B700CD008301CC008A45
:1058B00001920194012102230224022502260227DB
:1058C000022A02B300B4006F007000818283F76780
:1058D00066363534979694959392F637C6F5F4F17B
:1058E000303300010202020206060609090909090D
:1058F000090F0F0F0F0F0F15151518191919191971
:085900001919191919232400DB
:00000001FF
